:020000040000FA
:100000005AEF0CF01200FFFFC6EF03F01200FFFFE3
:10001000FFFFFFFFFFFFFFFFE6EF03F01200FFFF10
:10002000FFFFFFFFFFFFFFFFFFFF0100F8070000DA
:10003000EE00000005000000040120511F0B010824
:1000400001E05BD02051600BE842E842E842E84220
:10005000E842010801E051D0245103E0240501E009
:100060004CD02151230A48E0010A40E0030A30E065
:10007000010A25E0240A22E0070A1FE0010A1CE029
:10008000030A11E0010A01E038D00001030EE76F16
:100090000001D40EE86F000EE96F0001F493000137
:1000A000080EEC6F2AD00001030EE76F0001D40E9A
:1000B000EA6F000EEB6F21D020D01FD01ED00001C0
:1000C000030EE76F0001C90EEA6F000EEB6F15D04B
:1000D0000001030EE76F0001C90EE86F000EE96F23
:1000E0000001F4930001070EEC6F07D00001030E2E
:1000F000E76F22C4D0F001D000D012000001C96B1C
:10010000C20ECA6F010ECB6FCC6BCD6BCE6B080EDF
:10011000CF6FC26BC16B1A0E726E1E0E736E04012E
:10012000000E166F050E176F400E146F0401196F45
:10013000080E1A6F050E1B6F880E186F0401480E0B
:100140001E6F050E1F6F400E1C6F1200D9CFE6FF09
:10015000E1CFD9FF0001C16B040118BF30D0FC0E04
:10016000DBCF10F01951D880105403E2FC0E19C4F3
:10017000DBFF0001C16BFC0EDB50C15D19E2C15118
:10018000EA6A080FE96E050EEA22EF50E66EC151E9
:10019000E76EFD0EDBCFE9FFFE0EDBCFEAFFE75097
:1001A000E926000EEA22E552E750EF6EC12BE3D7B5
:1001B0000401400E196F1817187D880E18130001DE
:1001C000C15100D0E552E7CFD9FF1200D9CFE6FFE9
:1001D000E1CFD9FFE6520001C25101E02FD0DF6A22
:1001E000DF2ADF50106E116AFF0E101801E1115066
:1001F00001E10BD0FD0EDBCFE9FFDB2AFE0EDBCFEA
:10020000EAFF01E3DB2AEF50EBE1DF50106E116AE9
:10021000D950FD0FE96EFF0EDA20EA6E1050EE5E47
:100220001150ED5AFD0EDBCFC3F0FE0EDBCFC4F054
:10023000DFCFC7F00001C86B010EC26FE552E55277
:10024000E7CFD9FF1200D9CFE6FFE1CFD9FFE652C1
:100250000001C25101E030D0DF6ADF2ADF50106EAA
:10026000116AFF0E101801E1115001E10CD0FD0ED2
:10027000DBCFF6FFDB2AFE0EDBCFF7FF01E3DB2A45
:100280000800F550EAE1DF50106E116AD950FD0FF9
:10029000E96EFF0EDA20EA6E1050EE5E1150ED5A54
:1002A000FD0EDBCFC3F0FE0EDBCFC4F0DFCFC7F017
:1002B0000001010EC86FC26FE552E552E7CFD9FFCA
:1002C0001200D9CFE6FFE1CFD9FFE65204011CBFEF
:1002D0006BD0030E0001C25D01E1C26BC25101E1AE
:1002E00063D0020EC25D06E104011D6B0001030E26
:1002F000C26F54D0C20552E1400E106E116AC75150
:10030000105C000E115803E2400EDF6E02D0C7C031
:10031000DFFFDFCF1DF4DF50C75DC76F480EC56F2D
:10032000050EC66FC80515E1DF5012E0C3C0F6FF29
:10033000C4C0F7FF0800F550C5C0E9FFC6C0EAFF1A
:10034000EF6EC52B000EC623C32BC423DF06ECD7EC
:1003500013D0DF5011E0C3C0E9FFC4C0EAFFEF5083
:10036000C5C0E9FFC6C0EAFFEF6EC52B000EC6236D
:10037000C32BC423DF06EDD7C75110E104011D5183
:10038000106E116A400E101801E1115004E10001D5
:10039000020EC26F03D00001030EC26F400E0401B3
:1003A0001C171C7D880E1C13E552E552E7CFD9FFC0
:1003B000120004012051600BE842E842E842E842A2
:1003C000E842000901E055D02151070A51E00B0A2B
:1003D0004FE0070A40E0010A2CE00B0A28E0020A7D
:1003E00026E0030A22E0080A12E0010A0EE00F0AE2
:1003F0000AE0030A01E03CD00001010EE76F0001B2
:10040000040EF36F36D036D834D090D832D00001F5
:10041000010EE76F0001F50EE86F000EE96F0001B5
:10042000F4930001010EEC6F24D0A8D822D0F6D8A6
:1004300020D00001010EE76F040124510001E86F94
:10044000E96BF60EE827000EE9230001F4930001A2
:10045000010EEC6F0ED00001010EE76F0401245174
:10046000EA6AF60FE96E000EEA2222C4EFFF01D01D
:1004700000D01200800E0401205D57E12351030AD1
:1004800034E0010A10E0030A01E04DD00001010E42
:10049000E76F0001BE0EE86F060EE96F120E000155
:1004A000EC6FED6B40D00001010EE76F04012251AB
:1004B000F66EF76AD890F636F7367F0EF626070EF8
:1004C000F7220900F5CFE8F00A00F5CFE9F0020EB7
:1004D0000001F76AE825F66EE951F7220900F5CF29
:1004E000ECF00A00F5CFEDF01ED00001010EE76F31
:1004F00004012251F66EF76AD890F636F736830E6D
:10050000F626070EF7220900F5CFE8F00A00F5CF2E
:10051000E9F0E8C0F6FFE9C0F7FF0800F550000178
:10052000EC6FED6B00D00001F48312000001010EAE
:10053000E76F0F0EE66E710EE66E0F0EE66EB9EC0B
:100540000AF0E552E552E552010EE66EF60EE66E51
:10055000000EE66EB9EC0AF0E552E552E55222C40F
:10056000F5F00401225104E10001050EF36F05D0FE
:100570000001060EF36F7EEC00F012000401286B00
:10058000296B040120511F0B020A16E0030A10E038
:10059000010A01E035D00001010EE76F80A402D00E
:1005A000040128810001F4A102D00401288328D08D
:1005B0000001010EE76F24D00001010EE76F040176
:1005C00024510F0B080DF350116A000F106E040E2A
:1005D00011222451800B01E0010E040DF3500001A3
:1005E0001024EA6F000E1120EB6FEAC0E9FFEBC0A8
:1005F000EAFFEF50040B03E00401010E286F00D066
:100600000001E7050AE10001280EE86F040EE96F1A
:100610000001F4930001020EEC6F120004012205A8
:1006200010E120511F0B00090CE10001010EE76FE2
:10063000030E0401215D03E10001F48102D00001F9
:10064000F491040122513AE120511F0B020836E1D6
:1006500024510F0B000932E00001010EE76F040185
:1006600024510F0B080DF350116A000F106E040E89
:1006700011222451800B01E0010E040DF350000102
:100680001024EA6F000E1120EB6F030E0401215DB0
:1006900007E1840EEAC0E9FFEBC0EAFFEF6E0ED07F
:1006A00024AF06D0EAC0E9FFEBC0EAFFEF6A06D04C
:1006B000880EEAC0E9FFEBC0EAFFEF6E12001201FC
:1006C000000202000008D8040A0000000102000134
:1006D0000902430002010080320904000001020205
:1006E0000100052400100104240202052406000173
:1006F0000524010001070582030800020904010026
:10070000020A0000000705030240000007058302FB
:100710004000000403090434034D006900630072C3
:10072000006F0063006800690070002000540065DD
:1007300000630068006E006F006C006F0067007956
:1007400000200049006E0063002E00340343004483
:100750000043002000520053002D003200330032CD
:1007600000200045006D0075006C00610074006998
:10077000006F006E002000440065006D006F00D027
:1007800006D006130717074B073800FFDACFE4FF40
:10079000E2CFDAFFE9CFE4FFEACFE4FFE652F2A4CA
:1007A0000DD00001F95103E1F29406EC0CF00001C8
:1007B000F95104E0F2940001010EBE6FE552E5CF5D
:1007C000EAFFE5CFE9FFE5CFDAFF1100D8CFE4FF7C
:1007D000E0CFE4FFE46EDACFE4FFE2CFDAFFE652E7
:1007E000E552E5CFDAFFE550E5CFE0FFE5CFD8FFF2
:1007F00010004200410053000000000000FFFFFF16
:100800005AEF0CF01200939C9398939A939E936ADC
:100810008198819C819A819E0F0EC16E070EB46EE5
:10082000F19E948494829480929080909294929677
:100830009298929A808480868088808A0001A56937
:10084000A669A769A869BE6B8214BB6FBBC0BCF068
:100850000001F96B0001BF69010EC06FA06BA06BB6
:10086000400EA05D10E2A051EA6A030FE96E010E8E
:10087000EA22EF6AA051EA6A600FE96E000EEA22EE
:10088000EF6AA02BEDD70101006B0101016B0001A4
:10089000A26BA36BA16B090EB96F0C0EBA6F06EFBA
:1008A0000CF0060E0001F35D03E36D50020B01E056
:1008B00060D00001A35102E15DD85BD00001BE51C0
:1008C00003E090DA0001BE6B0001BF47010E00019A
:1008D000BF150001C01502E0010E01D0000E010B92
:1008E000F36EF346F346F346F346F346F346F34618
:1008F0007F0E8114F310816ED7EC0AF0800B01E0BB
:1009000038D006DA000901E134D00001C25131E1EA
:100910000001BD050BE1F60EE66E070EE66E23EC58
:1009200001F0E552E5520001BD6B23D0020E00013B
:10093000BD5D0BE1F40EE66E070EE66E23EC01F0F2
:10094000E552E5520001BD6B14D0030E0001BD5D00
:100950000BE1F20EE66E070EE66E23EC01F0E552B7
:10096000E5520001BD6B05D0EEEC0BF0000901E093
:100970008ED812000001A2510B0A01E181D0010AB8
:1009800001E17BD0030A6BE0010A5BE00F0A4BE058
:10099000010A3BE0030A2AE0010A25E0070A1CE0FD
:1009A000010A13E0030A0AE0010A01E06FD0D5BE94
:1009B00004D020EC0CF00001A22B68D0D5BE04D0EE
:1009C00020EC0CF00001A22B61D0D5BE04D020ECAD
:1009D0000CF00001A22B5AD0D5BE04D020EC0CF0B4
:1009E0000001A22B53D0D5AEA22B50D0D5BE0CD037
:1009F00020EC0CF0010EE66E200EE66E0AEC0BF019
:100A0000E552E5520001A22B41D0D5BE0BD020EC1F
:100A10000CF0E66A2C0EE66E0AEC0BF0E552E5529D
:100A20000001A22B33D0D5BE0BD020EC0CF0E66A2F
:100A3000BAC0E6FF0AEC0BF0E552E5520001A22B2A
:100A400025D0D5BE0BD020EC0CF0E66A010EE66E88
:100A50000AEC0BF0E552E5520001A22B17D0D5BEEF
:100A60000BD020EC0CF0E66A060EE66E0AEC0BF0FA
:100A7000E552E5520001A22B09D0D5AEA22B06D03B
:100A8000818E010EA36F28EC0CF000D01200000143
:100A9000A151120A01E19CD0030A01E194D0010A9C
:100AA00001E18DD01F0A01E186D0010A01E17FD06A
:100AB000030A01E17AD0010A73E0070A6DE0010A36
:100AC00067E0030A61E0010A5BE00F0A55E0010AF2
:100AD0004FE0030A49E0010A43E0070A2BE0010A5C
:100AE00022E0030A1EE0010A01E076D00101025172
:100AF000106E116AFE0E101801E1115005E002C1DE
:100B0000E6FF28EC0BF0E55201010251106E116A6C
:100B1000FE0E101801E1115003E10001010EA16F5A
:100B20005BD05BD859D0010102510001AC6FAD6BB5
:100B3000A12B52D0010102510001AE6FAF6BAEC0CC
:100B4000E6FFAFC0E6FFACC0E6FFADC0E6FF44EC99
:100B50000BF0E552E552E552E5520001A16B3CD0A5
:100B600002C1B0F0A12B38D002C1B1F0A12B34D01A
:100B700002C1B2F0A12B30D002C1B3F0A12B2CD016
:100B800002C1B4F0A12B28D002C1B5F0A12B24D012
:100B900002C1B6F0A12B20D002C1B7F0A12B1CD00E
:100BA00002C1B8F0B96BA16B17D0A16B15D0F4D905
:100BB0000001A16B11D012DA0001A16B0DD030DA67
:100BC0000001A16B09D002C1A4F0120EA16F04D0E4
:100BD00061DA0001A16B00D0120001010251FE0A8E
:100BE00001E18FD0660A01E188D0FE0A01E181D0DF
:100BF0003E0A75E00F0A6FE0010A69E0020A5BE055
:100C0000070A4DE0030A47E01E0A41E0050A33E007
:100C1000010A25E0020A19E00F0A13E0010A0CE0BC
:100C2000040A03E00001A16B72D0818E0001010E65
:100C3000C06F0D0EA16F6BD0819E0001C06BA16BC8
:100C400066D00001020EA16F62D0E66A020EE66E67
:100C50000AEC0BF0E552E5520001A16B58D00001FF
:100C6000BA83E66ABAC0E6FF0AEC0BF0E552E55239
:100C70000001A16B4CD00001BA93E66ABAC0E6FF4E
:100C80000AEC0BF0E552E5520001A16B40D00001E7
:100C9000040EA16F3CD000010D0EA16F38D00001F1
:100CA000BA81E66ABAC0E6FF0AEC0BF0E552E552FB
:100CB0000001A16B2CD00001BA91E66ABAC0E6FF30
:100CC0000AEC0BF0E552E5520001A16B20D00001C7
:100CD0000F0EA16F1CD000010E0EA16F18D0E66A96
:100CE000010EE66E0AEC0BF0E552E5520001A16B35
:100CF0000ED00001110EA16F0AD00001100EA16FDD
:100D000006D0FE0EE66E28EC0BF0E55200D0120085
:100D10000001B951090A60E0010A56E00F0A4CE0EF
:100D2000010A42E0030A38E0010A2EE0070A24E043
:100D3000010A1AE0030A10E0010A01E050D0E66A55
:100D4000080EB003F350400FE66E0AEC0BF0E552CC
:100D5000E5520001B92B43D0B1C0E6FF28EC0BF0FF
:100D6000E5520001B92B3BD0B2C0E6FF28EC0BF0F6
:100D7000E5520001B92B33D0B3C0E6FF28EC0BF0ED
:100D8000E5520001B92B2BD0B4C0E6FF28EC0BF0E4
:100D9000E5520001B92B23D0B5C0E6FF28EC0BF0DB
:100DA000E5520001B92B1BD0B6C0E6FF28EC0BF0D2
:100DB000E5520001B92B13D0B7C0E6FF28EC0BF0C9
:100DC000E5520001B92B0BD0B8C0E6FF28EC0BF0C0
:100DD000E5520001B92B03D0010E03D000D0000E64
:100DE00000D012000001AA070001AA5165E100012C
:100DF000960EAA6F0001A5470001A6470001A7476C
:100E00000001A847010E0001A915106E010E000196
:100E1000A5151002F35002E0010E01D0000E010BE7
:100E2000F36EF346F346FB0E8014F310806E020E51
:100E30000001A915106E010E0001A6151002F35055
:100E400002E0010E01D0000E010BF36EF346F346F3
:100E5000F346F70E8014F310806E040E0001A915FE
:100E6000106E010E0001A7151002F35002E0010EF2
:100E700001D0000E010BF36EF346F346F346F34642
:100E8000EF0E8014F310806E080E0001A915106E8D
:100E9000010E0001A8151002F35002E0010E01D06E
:100EA000000E010BF36EF346F346F346F346F346AA
:100EB000DF0E8014F310806E0001AB070001AB5110
:100EC0006AE10001320EAB6FBBC0BCF0070E8214AA
:100ED0000001BB6F0001BB510001BC5D5CE0040E72
:100EE0000001BB15040802E0000E01D0010E116ED6
:100EF000040E0001BC15106E040E0001BB15105C41
:100F000002E1000E01D0010E11140CE00001BBA3A0
:100F100005D00001020EBD6F3ED004D00001030ECB
:100F2000BD6F39D0040E0001BB15040802E1000EAC
:100F300001D0010E116E040E0001BC15106E040EDE
:100F40000001BB15105C02E1000E01D0010E11146E
:100F50000CE00001BBA305D00001030EBD6F1BD048
:100F600004D00001020EBD6F16D0010E0001BB15AA
:100F7000116E010E0001BC15106E010E0001BB15B3
:100F8000105C02E1000E01D0010E111404E000011A
:100F9000010EBD6F00D0120001010251050A19E0D7
:100FA000010A13E0070A0DE0010A07E0030A01E065
:100FB00012D080840001A98110D080860001A9830D
:100FC0000CD080880001A98508D0808A0001A987FB
:100FD00004D0808002D0000000D012000101025134
:100FE000050A19E0010A13E0070A0DE0010A07E00B
:100FF000030A01E012D080940001A99110D08096DC
:101000000001A9930CD080980001A99508D0809A7E
:101010000001A99704D0809002D0000000D01200F7
:101020001F0E106E10C00CF002C107F04CEC0CF05B
:1010300007C0BFF00001BF51080A29E00F0A24E0F1
:10104000010A1FE0030A1AE0010A15E0070A10E08E
:10105000010A0BE0030A06E0010A02E0BF6919D0A9
:10106000BF6B17D0010EBF6F14D0110EBF6F11D020
:10107000910EBF6F0ED0550EBF6F0BD0570EBF6FC6
:1010800008D0EE0EBF6F05D0FE0EBF6F02D0BF6955
:1010900000D012000C0E106E10C00CF002C107F050
:1010A0004CEC0CF007C002F101010251080A29E0E2
:1010B0000F0A24E0010A1FE0030A1AE0010A15E002
:1010C000070A10E0010A0BE0030A06E0010A02E049
:1010D000026919D0026B17D0010E026F14D0110EE5
:1010E000026F11D0910E026F0ED0550E026F0BD011
:1010F000570E026F08D0EE0E026F05D0FE0E026F83
:1011000002D0026900D00001A451040A10E0070ACD
:101110000BE0010A06E0030A01E00CD002C1A5F0D1
:1011200009D002C1A6F006D002C1A7F003D002C1C7
:10113000A8F000D012006C5002E0000E01D0010EA9
:1011400000090BE0040100513C0BE842E8420D08A5
:1011500002E10CD801D040D808D06C5002E0000E5B
:1011600001D0010E040901E047D81200D9CFE6FFF3
:10117000E1CFD9FFE6520001E66BE76BEC6BED6B5C
:10118000D9EC01F0DF6ADF50106E116A010E105CBD
:10119000000E11581BE20001E75101E017D0F76A79
:1011A000DF34FE0BF736F66E890EF626070EF722B1
:1011B0000900F5CF10F00800F5CF11F004D011C0F0
:1011C000FAFF1050F96EFBDFDF2ADDD7D5D8E552E4
:1011D000E552E7CFD9FF1200020E0001E65D0AE1F9
:1011E00092D8040100BD03D0C80E006F02D0880E53
:1011F000006F01D007D91200040E0001F35D0AE16F
:1012000022C46EFF6E50000803E2050EF36F02D099
:10121000030EF36F0001E6050AE10BD8040104BDDB
:1012200003D0C80E046F02D0880E046F01D0EAD834
:101230001200D9CFE6FFE1CFD9FF020EE12600016F
:10124000080EEC5D000EED5905E2ECC0DEFFEDC0CE
:10125000DDFF03D0080EDE6EDD6A04010493049105
:10126000010EDB500413DFCF05F4000EDB5000014C
:10127000EC5F010EDB50ED5B280EEA6F040EEB6FA6
:101280000001F4A31ED0D9CFE9FFDACFEAFFEE5078
:10129000ED1016E0E8C0F6FFE9C0F7FF0800F550D2
:1012A000EAC0E9FFEBC0EAFFEF6E0001EA2B000E97
:1012B000EB23E82BE923DF06010E01E2DB06E3D78F
:1012C0001CD0D9CFE9FFDACFEAFFEE50ED1015E0E0
:1012D000E8C0E9FFE9C0EAFFEF50EAC0E9FFEBC070
:1012E000EAFFEF6E0001EA2B000EEB23E82BE92367
:1012F000DF06010E01E2DB06E4D7D9CFE1FFE552BC
:10130000E7CFD9FF1200D9CFE6FFE1CFD9FF020E18
:10131000E126030E04010015E76E010EE7CFDBFFA7
:1013200001C4DFFFDE500001EC27DD50ED23280E65
:10133000E86F040EE96FD9CFE9FFDACFEAFFEE508C
:10134000ED1014E0E8C0E9FFE9C0EAFFEF50EAC0A1
:10135000E9FFEBC0EAFFEF6EEA2B000EEB23E82B70
:10136000E923DF06010E01E2DB06E5D7D9CFE1FF75
:10137000E552E7CFD9FF12000001E7510CE104016B
:10138000080E016F200E026F040E036F840E006FB3
:101390000401046F35D0040120AF22D00001EC51CC
:1013A0000401265D0001ED510401275904E226C421
:1013B000ECF027C4EDF03DDF0001010EE66F040103
:1013C000080E016F200E026F040E036F800E006F77
:1013D0000401280E066F040E076FC80E046F10D0AC
:1013E0000001020EE66F0401056BC80E046F0401D4
:1013F000080E016F280E026F040E036FC80E006FF7
:101400006D9812000001E66B0401080E016F200EBA
:10141000026F040E036F880E006F0401046B12004C
:101420006DA60FD802D06DB613D80001F30508E100
:101430006DBA06D0686A696A69806988020EF36FBE
:1014400012006D6A696A6D860001010EF36F120069
:101450006D6A696A0001F36B120028EF0AF000015F
:10146000F35101E13AD06850040B04E06950040BD9
:1014700001E03CD86DB231D06850010B04E06950F6
:10148000010B01E054D86850100B04E06950100BB8
:1014900001E024D86850400B04E06950400B01E0A3
:1014A0003BD86850200B04E06950200B01E036D88F
:1014B0006850020B04E06950020B01E036D8030EBD
:1014C0000001F35D01E209D06850080B06E06950A5
:1014D000080B03E09BEC08F068961200698468989A
:1014E0006D82A19AA08A0300A09A12006D9269945D
:1014F000689412000001F4A10ED0F8DF6D840001A1
:10150000080EF76F070EF86FF707000EF85BF7513C
:10151000F811FAE16D941200689C120070A003D0DB
:1015200002EC0AF07090689A1200689212006A6ADF
:10153000686A9F0E6B6E7B0E696E6E6A0F0EE66EAA
:10154000710EE66E0F0EE66E14D8E552E552E552C6
:10155000160E706E68A602D06896FCD76D9802ECE5
:101560000AF00001F4910001F56B0001030EF36F26
:101570001200D9CFE6FFE1CFD9FFFD0EDBCFE9FFA7
:10158000FE0EDBCFEAFFFC0EDB5004E0EE6AFC0E41
:10159000DB06F9D7E552E7CFD9FF120081880000BA
:1015A0000000000000000000000081981200800E82
:1015B000811402E0010E01D0000E0001FA6F816A71
:1015C0000F0E936E819C818A8188000000000000CC
:1015D00000000000000081CFEEF081980001EE399C
:1015E000F00BF00B0001EE6F81880000000000009E
:1015F0000000000000000F0E81100001EE13819822
:10160000819A936A0001FA5101E0818E0001EE5146
:1016100000D01200D9CFE6FFE1CFD9FF819C819A9B
:10162000F00E8116FE0EDB380F0B0F0B8112B6DFAA
:10163000FD0EDB5007E1F00E8116FE0EDB500F0BA6
:101640008112ACDFF00E8116E552E7CFD9FF120010
:10165000D9CFE6FFE1CFD9FF818C819AF00E8116B8
:10166000FE0EDB380F0B0F0B811298DFF00E811688
:10167000FE0EDB500F0B811291DFF00E8116819C64
:10168000E552E7CFD9FF1200D9CFE6FFE1CFD9FF6E
:10169000FB0EDBCF06F0FC0EDBCF07F0040E0618C6
:1016A00001E107501CE0030E061801E1075013E0AA
:1016B000020E061801E107500AE0010E061801E1CA
:1016C000075001E010D00001800EEF6F0CD0000138
:1016D000C00EEF6F08D00001940EEF6F04D0000130
:1016E000D40EEF6F00D0FD0EDBCF10F0FE0EDBCF7F
:1016F00011F01006000E115A10500001EF27E66A93
:10170000EFC0E6FF87DFE552E552E552E7CFD9FFAC
:1017100012002A0EF66E000EF76E000EF86E000133
:101720000900F550E16F0900F550E26F03E1E16750
:1017300001D03DD00900F550DC6F0900F550DD6F98
:101740000900F550DE6F09000900F550E96E090047
:10175000F550EA6E090009000900F550DF6F090035
:10176000F550E06F09000900F6CFE3F0F7CFE4F0A1
:10177000F8CFE5F0DCC0F6FFDDC0F7FFDEC0F8FF14
:101780000001DF5302E1E05307E00900F550EE6E7F
:10179000DF07F8E2E007F9D7E3C0F6FFE4C0F7FFA0
:1017A000E5C0F8FF0001E107000EE25BBFD71200C1
:1017B000400EE66E030EE66E010EE66EA6EC00F03D
:1017C000E552E552E552000906E0C1C001F1010110
:1017D000006B010E02D0000E00D01200010100517A
:1017E000D880015507E3E4DF000902E1000E0DD0C7
:1017F0000101006B0051EA6A030FE96E010EEA2253
:10180000EFCF02F1002B010E00D01200F29A7F0EF2
:10181000D56E1200D9CFE6FFE1CFD9FFFE0EDB5027
:101820007F0BD56ED76AD66AF294FE0EDBAE02D07D
:10183000F28A01D0F29AD58EE552E7CFD9FF120095
:10184000D08EC00EF212D70EE66EE4DFE552120023
:10185000D08EC00EF2120001010EF96FD20EE66EAC
:10186000D9DFE552120005D80FD851EC04F0FCD7AF
:1018700012009284140E6F6E0001F36B0001F46B82
:101880000001F56B03EF04F010EC0AF06FBE02D01C
:101890002FEC0AF061EF01F0036A080EE76ED890B2
:1018A000073603360C50035C02E3036E072AE72E6B
:1018B000F7D7120013EE00F023EE00F0F86A0F9C49
:1018C00089EC0BF033EC0CF0FDD71200FFFFFFFFAB
:1018D000FFFFFFFFFFFFFFFFFFFFFFFFFFFFFFFF18
:1018E000FFFFFFFFFFFFFFFFFFFFFFFFFFFFFFFF08
:1018F000FFFFFFFFFFFFFFFFFFFFFFFFFFFFFFFFF8
:10190000FFFFFFFFFFFFFFFFFFFFFFFFFFFFFFFFE7
:0200000400F00A
:020000040030CA
:0E00000020033E1E008181000FC00FE00F4064
:00000001FF
